:100000003CC054C054C052C051C050C04FC04EC07C
:1000100059C04CC04BC04AC049C048C047C046C088
:1000200045C00E0304000F060501080A090B0D0761
:100030000C021011121337C89F209F6017E8E718B1
:100040001FE06F90F708B748CF304FB0EF100FF0B8
:100050003FC05FA0D7282FD00000000000005069EB
:100060006C6F7420562D4D6174652056312E3020F2
:100070002863294D69736975200011241FBECFEDD7
:10008000CDBF10E0A0E6B0E0ECE1F4E003C0C8951D
:1000900031960D92A036B107D1F710E0A0E6B0E09E
:1000A00001C01D92A036B107E1F742C1A9CF1F924E
:1000B0000F920FB60F92112400000F900FBE0F90F9
:1000C0001F9018951F920F920FB60F9211241EBC0D
:1000D0001CB80F900FBE0F901F9018952EE130E0C6
:1000E000281B390B3DBD2CBD81E08BB98CB98EBD71
:1000F00080E285BF8EB5882319F088950000FACF7D
:1001000008959F92AF92BF92CF92DF92EF92FF92AB
:100110000F931F93CF93A62EB72EC82ED92E942EB1
:1001200020EFE22E2BECF22E27E8022F26E0122FF2
:10013000C298BA98C09A10BE13BE8CE390E0CEDF8E
:10014000B09906C08DE086BF83E480BF89E083BF9D
:10015000C098BA9A80E692E2C1DFBA9880E391E152
:10016000BDDF9920D9F4C92DBA9A8CE192E0B6DFAF
:10017000CA3121F41B2D0A2DFF24EE24BA9817FF53
:1001800003C088E696E002C08CE192E0A7DFEE0CA7
:10019000FF1C001F111FCF5FCA3230F3BA9A86E2EC
:1001A00092E09CDFBA9810BE13BE992019F08CED36
:1001B0009FEF94DF88EC92E391DFCF911F910F9135
:1001C000FF90EF90DF90CF90BF90AF909F900895F9
:1001D000FF920F931F93CF93F82EC0E00C2F10E0E7
:1001E0000ABB802F80958BBB82E390E077DFC89BB2
:1001F00011E0C99B12E0CA9B13E0CF9902C014E042
:1002000008C0112331F4000F09F408E0CF5FC530B6
:1002100030F31ABA8FEF8BBB112301F1CC2309F411
:10022000C5E0C150CC0FCC0FC10FC150AC2FBB27C4
:10023000FF2021F08A2F9B2F019612C0DBD0802D4A
:10024000843160F4E82FFF27EE0FFF1FEA5CFF4FB9
:10025000C895802D3196C895902D02C080E090E021
:10026000CF911F910F91FF900895CF939DE096BF7E
:1002700093E490BF99E093BFC82FC150CF3FA9F03E
:10028000BA9A88EE9DEF2ADF88EE9DEF27DFBA98B5
:1002900088EE9DEF23DF88EE9DEF20DF88EE9DEF57
:1002A0001DDF88EE9DEF1ADFE8CF10BE13BECF91A1
:1002B0000895DF92EF92FF920F931F93CF93DF93F6
:1002C00000E0D02E48EBE42E4BE0F42E86E0CDDFAC
:1002D00081E07EDFD92FC82F80E197E2FFDECC23BB
:1002E000A9F0CD1599F081E073DFC81779F4DC2E01
:1002F000AC2FBB271197002E85D0802F83708F5F86
:10030000B4DF0F5F38EBE32E3BE0F32E0894E108F7
:10031000F108013118F4E114F104D1F686E0A5DF0B
:10032000DF91CF911F910F91FF90EF90DF90089593
:10033000CFEDD0E0DEBFCDBFF8948AEF88BB17BA0F
:100340008FEF8BBB1ABA80E888B916B883E080B902
:1003500087E882BB80E18ABF8BBF7894B19905C0E2
:1003600080E593ECBBDEB19BA4DF10E0A12FBB279F
:100370002A2F3B2F3FD0802D843150F0F32FE22FD6
:10038000EE5DFF4FC895802DB32FA22F082E3AD0D7
:100390001F5F143158F388E78ABB87E88BBB8FE077
:1003A00080B980E385BF88950000000080E29EE46C
:1003B00095DE83E080B912E380E00ADFD92FC82FF1
:1003C000892B49F380E197E289DE80E001DFC817DD
:1003D000D90709F740E0123309F041E08C2F9D2F37
:1003E000AA27BB27682F792F8A2F9B2F8ADE1150CF
:1003F00019F7D1CFE199FECFBFBBAEBBE09A119602
:100400000DB20895E199FECFBFBBAEBB0DBA1196F8
:0C0410000FB6F894E29AE19A0FBE08952E
:00000001FF
